:100000000C945F030C9497030C9497030C94970340
:100010000C9497030C9497030C9497030C949703F8
:100020000C9497030C9497030C947D260C945527FD
:100030000C9432260C9497030C9497030C9497031A
:100040000C9497030C9497030C9497030C949703C8
:100050000C9497030C9459260C9497030C949703D3
:100060000C9497030C9497030C9497030C949703A8
:100070000C9497030C9497030C9497030C94970398
:100080000C9497030C9497030C9497030C94970388
:100090000C9497030C9497030C9497030C94970378
:1000A0000C9497030C9497030C9497030501098013
:1000B000A101850319012AB700150126B700950192
:1000C00075108100C0050C0901A101850419012AE0
:1000D000A002150126A002950175108100C00660DE
:1000E000FF0961A1010962150026FF00952075082E
:1000F00081020963150026FF00952075089102C052
:1001000005010906A101050719E029E715002501E8
:10011000950875018102950175088101050719008F
:1001200029FF150026FF00950675088100050819AE
:10013000012905950575019102950175039101C08D
:100140000E018466FFFF000000000F018466FFFFC0
:100150000000000010018466FFFF000000000301A2
:100160008466FF0A0155FFFF120155FFFFFF0000E3
:10017000000004018466FF090155FFFF130155FFCC
:10018000FFFF0000000011018466FF180155FFFF0A
:10019000FF000000000B018466FFFF000000001458
:1001A000018466FF0C0155FFFFFF000000000902FB
:1001B0005B00030100A0FA09040000010301010033
:1001C00009211101000122400007058103080001F7
:1001D00009040100020300000009211101000122AD
:1001E0002200070582032000010705030320000108
:1001F000090402000103000000092111010001228D
:1002000032000705840320000112010002000000F3
:1002100008F1F125000100010200011603570069F1
:10022000006E007200790020003200350074006614
:100230000000001A0353007000690064006500723A
:1002400000490073006C0061006E0064000000044F
:10025000030904530054005500560029005F006054
:10026000006100570020785C005D005E00580021AE
:100270007859005A005B005200215262006300501E
:100280000051004F002078217822782B782378279E
:10029000782578237829782C782878267824782A65
:1002A000780000625263526452000000006552669A
:1002B0005267520000000000000000000000000033
:1002C00000000000005A00000000000000000000D4
:1002D00000000000000000000000000000005200CC
:1002E000000000000000000000000000000000000E
:1002F000000000000000005B0000000000000000A3
:1003000000000000000000000000000000000000ED
:10031000520000000000000000000000000000008B
:100320000000000000000000005C00000000000071
:1003300000000000000000000000000000000000BD
:10034000000052000000000000000000000000005B
:1003500000000000000000000000005D0000000040
:10036000000000000000000000000000000000008D
:10037000000000005200000000000000000000002B
:10038000000000000000000000000000005E00000F
:10039000000000000000000000000000000000005D
:1003A00000000000000052000000000000000000FB
:1003B0000000000000000000000000000000005FDE
:1003C000000000000000000000000000000000002D
:1003D00000000000000000005200000000000000CB
:1003E0000000002223252628292A2C2D2F303233E5
:1003F0003536383A3B3D3E4042434547494A4C4EEC
:100400005051535557595A5C5E6062646668696B17
:100410006D6F71737577797B7D7F81838587898A1D
:100420008C8E90929496989A9C9E9FA1A3A5A7A823
:10043000AAACAEAFB1B3B4B6B8B9BBBCBEBFC1C253
:10044000C3C5C6C7C9CACBCCCDCED0D1D2D2D3D4E6
:10045000D5D6D7D7D8D9D9DADADBDBDBDCDCDCDC04
:10046000DCDDDDDDDDDCDCDCDCDCDBDBDBDADAD9D2
:10047000D9D8D7D7D6D5D4D3D2D2D1D0CECDCCCB54
:10048000CAC9C7C6C5C3C2C1BFBEBCBBB9B8B6B472
:10049000B3B1AFAEACAAA8A7A5A3A19F9E9C9A9802
:1004A000969492908E8C8A89878583817F7D7B79D3
:1004B000777573716F6D6B6968666462605E5C5AB4
:1004C0005957555351504E4C4A4947454342403E77
:1004D0003D3B3A3836353332302F2D2C2A29282609
:1004E000252322FFAA7F55400001010101010101DE
:1004F00001010202020202020202020303030303D9
:1005000003030304040404040404050505050506A7
:100510000606060607070707070808080809090965
:10052000090A0A0A0B0B0B0C0C0C0D0D0D0E0E0E0E
:100530000F0F0F101011111112121313141415159F
:1005400016161717181819191A1A1B1B1C1D1D1E11
:100550001E1F202021222223242425262627282965
:10056000292A2B2C2D2D2E2F303132323334353693
:100570003738393A3B3C3D3E3F4041424344454693
:100580004748494A4C4D4E4F50515354555658596F
:100590005A5B5D5E5F616264656668696B6C6D6F16
:1005A0007072737577787A7B7D7E80828385878889
:1005B0008A8C8E8F91939596989A9C9EA0A2A3A5C3
:1005C000A7A9ABADAFB1B3B5B7BABCBEC0C2C4C6C4
:1005D000C9CBCDCFD1D4D6D8DBDDDFE2E4E7E9EB80
:1005E000EEF0F3F5F8FAFDFF9F0195018601720127
:1005F0005E0154014A01400100001E0F057F3F1FAC
:10060000643214643214783C1E1E140A0500000083
:1006100000000000000000000000000000000000DA
:1006200000000000000000000000000000000000CA
:10063000007E0F00D4FFFFFFC7000000780000001D
:1006400000000000002A2B2800000000000000002D
:10065000000000000000000029000000002C1E34F3
:1006600020212224342627252E362D3738271E1FF9
:10067000202122232425263333362E37381F040524
:10068000060708090A0B0C0D0E0F10111213141592
:10069000161718191A1B1C1D2F3130232D35040570
:1006A000060708090A0B0C0D0E0F10111213141572
:1006B000161718191A1B1C1D2F3130354C00112428
:1006C0001FBECFEFDAE0DEBFCDBF04B603FE18C019
:1006D00080916E0390916F03A0917003B0917103AC
:1006E0008730904BA740B04B59F410926E03109294
:1006F0006F031092700310927103E0E0F8E3099524
:1007000023E0A4E9B1E001C01D92AE36B207E1F7E3
:1007100011E0A0E0B1E0E8EBF3E502C005900D9236
:10072000A439B107D9F70E94BC210C947F290C94FD
:100730000000809330030895292F953098F5853077
:1007400088F590E035E0239F800D911D1124282F1E
:10075000277041E001C0440F2A95EAF723E09695FF
:1007600087952A95E1F7FC01EE0FFF1FE80FF91FAF
:10077000EA50FD4F20E030E070E05191DF01119729
:10078000CB01022E02C0969587950A94E2F78170FC
:1007900081958527842385278C932F5F3F4F2330B6
:1007A000310559F70895292F953078F5853068F58A
:1007B00090E035E0239F800D911D1124682F677014
:1007C00023E0969587952A95E1F7FC01EE0FFF1F30
:1007D000E80FF91FEA50FD4F40E050E080E0219122
:1007E00030E0062E02C0369527950A94E2F7217074
:1007F0003327042E01C0220F0A94EAF7822B4F5FA1
:100800005F4F4330510559F7089580E00895809176
:10081000370390913603981301C008958F5F877056
:10082000FACFE8E9F1E09191891303C0DF01119754
:100830001C9291E0EE39F907B1F70895982F909541
:1008400080912E03892380932E03089580912F0396
:10085000811110922F030895803E9105D1F1C8F4C3
:100860008133910509F47FC048F48932910509F478
:100870006FC08A32910509F47DC0089589339105CE
:10088000E1F082389105C9F08533910509F45BC028
:100890000895843E9105D1F148F4823E910531F1ED
:1008A000833E910541F181EE90E00895863E9105E9
:1008B000C1F1873E9105E1F1089520913303237042
:1008C000211165C02091340323FF14C089E290E018
:1008D00008952091330320FD43C03091340330FF4D
:1008E00009C024FF4EC080E090E0089520913303BA
:1008F00022FDF7CF08952091330322FD45C03091AA
:10090000340330FD44C024FFF5CFEDCF20913403F4
:1009100021FFF0CF8091330384FDE5CF87EE90E097
:1009200008952091330323FFE5CF24FDDCCFF6CFDC
:100930002091330323FD2EC03091340331FFE3CFE8
:1009400084EE90E008952091330325FFD3CFBECFEE
:100950002091330325FD21C02091340323FFCACF0A
:1009600089E390E008952091330326FFC3CF8AE204
:1009700090E008952091330326FFBCCF81E390E0FF
:10098000089583EE90E0089582EE90E0089580EE61
:1009900090E0089586EE90E0089585E390E0AACF78
:1009A0002091330322FF06C0982F98719830C1F42C
:1009B000877F846090913403392F3170927023FFC8
:1009C00021C0482F4871483191F4877E8461992372
:1009D000B1F0982F9171913191F48E7E88610FC0A2
:1009E000982F9471943031F78B7F8860E3CF482F34
:1009F0004471443139F48B7E8861911118C024FD13
:100A0000877E0895332369F0382F3871383019F410
:100A1000877F8160DCCF382F3171313011F48E7FC8
:100A20008860992361F3982F9871983191F6877EA9
:100A30008161E5CF1F93CF93DF930E942C04EC01DB
:100A4000811522E5920708F053C0811540E594070F
:100A500008F0DDC0803E9105F8F48D3C910508F06A
:100A6000AEC0883A910580F4853A910508F099C0A6
:100A70008130910521F00497813A910550F4CE011F
:100A8000DF91CF911F910895885A91094B9708F4EF
:100A90008BC0C0E0D0E0F3CF811550E49507F8F4A7
:100AA000C11580E2D80708F0CBC0C83ED10538F3A5
:100AB000CE019A9581159F4160F78D2F0E94D00439
:100AC000182FCE0199270E942C04212F30E0322FBD
:100AD0002227E901CC27DF71C82BD92BD0CF99274A
:100AE0000E942C04CC27DF70C82BD92BD06AC7CF2B
:100AF000803842E59407C8F5803652E5950708F03E
:100B000067C0C03482E5D807B0F08C2F86958695F3
:100B1000877020E2829FC0011124C37021E030E081
:100B2000A90102C0440F551FCA95E2F7EA01C82B7C
:100B3000D92BDC68A4CFC03252E5D50708F041C0FC
:100B40008C2F8695869520E2829FC0011124C37068
:100B500021E030E0A90102C0440F551FCA95E2F719
:100B6000EA01C82BD92BDD688ACF803C52E5950776
:100B700060F48F71C03AD24508F03FC090E0982FE2
:100B80008827EC01C46FD06A7ACF805C9245809749
:100B900008F07FCFDC2FCC27CC27DF71C06FD06A65
:100BA0006ECFA497D0646BCFC85AD0E0CC0FDD1FB6
:100BB000C35ADE4F0990D881C02DD46460CFD06570
:100BC0005ECFCF71D0E0DC2FCC27C16FD06A57CF7A
:100BD00086958695877020E2829FC0011124C3709C
:100BE00021E030E0A90102C0440F551FCA95E2F789
:100BF000EA01C82BD92BDA6842CF0E94D004C82F53
:100C0000D0E0DC2FCC27CC27DF71D06238CF8F71BA
:100C10000E94D00465E0D695C7956A95E1F7CF703C
:100C2000D0E0DC2FCC27282F30E084FF05C054E033
:100C3000220F331F5A95E1F7C22BD32BD0691FCF58
:100C40008D2F8F710E94D004182FCE0199270E94FA
:100C50002C04212F30E0322F222722273F71282B0E
:100C6000392BE901D2CF80E00895F894E82FE2957E
:100C7000EF70F0E041A18F7021E030E0B90102C0D7
:100C8000660F771F8A95E2F7CB01962F90959423F4
:100C900091A392A1892B82A3789408950895A0E04E
:100CA000B0E0E5E5F6E00C940428E901E42FF0E07B
:100CB000E851FB4F61110BC0E4919E2F8E2F898369
:100CC000E8839A83CDB7DEB7EAE00C942028282F7A
:100CD00030E0062F10E0F491EF2F86E0829F600154
:100CE000839FD00C1124EE24EA94F12CC601B701A5
:100CF0000E94B827220F331F45E5469FC001479F3A
:100D0000900D1124281B390B822F880F280FC70143
:100D1000801B910BF89FA001F99F500D1124952F76
:100D2000209F5001219FB00C1124AB2CBB24D70174
:100D3000AA19BB095D01FA9DD001FB9DB00D1124DC
:100D40008B2F5701A21AB1089501209F5001219FB6
:100D5000B00C309FB00C1124AB2CBB24EA18FB085C
:100D6000FE9D9001FF9D300D112463307105C9F087
:100D70001CEFC11613E0D10650F46130710509F47F
:100D80009ECF6230710589F08E2FE32F98CF6430AB
:100D9000710571F066307105B9F3E52F9B2F8F2F28
:100DA0008ECFEB2F852F9F2F8ACF852F932F87CF25
:100DB000832FE52FF8CF80912903823060F4817072
:100DC00082608093290380912C03873918F086E98B
:100DD00080932C0308958235B0F381708065F1CF44
:100DE00021E030E0A90102C0440F551F8A95E2F7C7
:100DF000CA012091270330912803662351F0242B48
:100E0000352B309328032093270381E08093DC0265
:100E100008958095909528233923F3CF682F61702A
:100E200080E00E94F0060895FA01882311F00995E8
:100E30000895FB01FCCFE091EC02F091ED023097B8
:100E400029F00190F081E02D0995089580E0089542
:100E50001F93CF93DF93182F0E941B07682F617099
:100E600080E00E94F006111121C060E081E00E9444
:100E7000F00660E082E00E94F00660E083E00E94FD
:100E8000F00660E084E00E94F00660E085E00E94E9
:100E9000F00660E086E00E94F00660E087E00E94D5
:100EA000F006812FDF91CF911F910895C12FD0E0DF
:100EB000BE0175956795617081E00E94F006BE01E4
:100EC0007595679575956795617082E00E94F0064B
:100ED000BE0123E0759567952A95E1F7617083E07F
:100EE0000E94F006BE0134E0759567953A95E1F7EA
:100EF000617084E00E94F006BE0145E0759567953B
:100F00004A95E1F7617085E00E94F006BE0156E067
:100F1000759567955A95E1F7617086E00E94F00635
:100F2000CC0FCD2FCC1FDD0B6C2F6170B7CF0E9483
:100F3000280780933103089521E030E001C0220F9B
:100F40008A95EAF780913103822B0E9497070895D2
:100F500021E030E0A90102C0440F551F8A95E2F755
:100F6000CA0180959091310389230E9497070895C3
:100F7000209132038095822380933203982F9770BB
:100F8000911113C030E0482F082E000C550B241788
:100F9000350759F09091340392FF07C085958595E8
:100FA00085950E94A807109232030895909131030D
:100FB00021E030E0F90101C0EE0F8A95EAF7D9018E
:100FC00002C0AA0FBB1F6A95E2F7EA2B01C0220FED
:100FD0004A95EAF7892F8E23E81305C0892F822BC3
:100FE0000E94970708952095822F8923F9CFA3E0C7
:100FF000B0E0EDEFF7E00C940C289C018091BE016D
:101000009091BF0182179307A1F03093BF01209305
:10101000BE01E091EC02F091ED02309751F083E0D7
:1010200089833B832A830680F781E02DCE010196D8
:1010300009952396E2E00C942828A3E0B0E0E3E2CF
:10104000F8E00C940C289C018091BC019091BD01AA
:1010500082179307A1F03093BD012093BC01E0916A
:10106000EC02F091ED02309751F084E089833B83EC
:101070002A830680F781E02DCE01019609952396FB
:10108000E2E00C9428289C01FC0132968FEF90E05E
:101090004191461751F08F3F19F4411101C0892F3A
:1010A0009F5F9630A9F78F3F09F40895280F311DEF
:1010B00087FD3A95F901628308952FB7F8948091DE
:1010C000B8019091B901A091BA01B091BB012FBFB5
:1010D0000895A4E0B0E0EFE6F8E00C940C288FB798
:1010E000F8942091B8013091B9014091BA01509122
:1010F000BB0129833A834B835C838FBF69817A81EB
:101100008B819C812496E2E00C9428288091B70181
:1011100008950895FC019B018091AD019091AE016D
:101120008617970740F0672B29F48091E8008E77A7
:101130008093E800C90140E0009741F4411106C0E6
:101140008091E80082FF2FC080E008952091E9029D
:101150002223A9F12530A9F12091E80023FD2DC01B
:101160002091E80022FDECCF2091E80020FFE4CFA1
:101170003091F3002091F200009719F028303105EA
:1011800058F041E02830310509F040E02091E800B6
:101190002E772093E800D0CF41914093F100019742
:1011A0002F5F3F4FE9CF8091E902882341F08530DE
:1011B00041F08091E80083FFC3CF81E0089582E091
:1011C000089583E008958091A70187FF13C080915F
:1011D000E80082FF06C08091E8008B778093E800EA
:1011E00004C08091E9028111F2CF08958091E90253
:1011F0008823D9F38091E80080FFF8CF8091E80040
:101200008E77ECCF2091E4003091E50095E6A901BE
:101210008091EC008170882331F08091E80080FF9C
:1012200006C080E008952091E80022FD1BC0809157
:10123000E902882391F0853091F08091EB0085FDE3
:1012400010C02091E4003091E5004217530701F3EC
:1012500091509111DCCF84E0089582E0089583E0FD
:10126000089581E00895E8EDF0E080818E7F80832D
:101270001092E2001092DA001092E100A0EEB0E0CD
:101280008C9181608C9380818F77808319BCA7EDCE
:10129000B0E08C918E7F8C9380818F7E80831092C2
:1012A000A6010895982FE42FE2709093E900891326
:1012B00008C0762F242F50E0E11111C091E0980F63
:1012C000F4CF7091EC002091ED005091F00021FDE1
:1012D00006C09F5F973049F78093E90008953091E9
:1012E000EB003E7F3093EB003091ED003D7F30937B
:1012F000ED003091EB0031603093EB007093EC0027
:101300002093ED005093F0002091EE0027FDE1CFF7
:101310000895A0E0B0E0EFE8F9E00C940628C8EDED
:10132000D0E088818F7E8883E7EDF0E08081816066
:10133000808384E082BF81E08093A60188818E7FD4
:10134000888302EE10E0F80110821092DA0081EE3C
:10135000C82ED12CF601108288818F7788838881EE
:101360008068888388818F7D888319BC1092E90208
:101370001092A5011092D5021092A40190EEE92ED0
:10138000F12CF70180818B7F808388818160888345
:1013900042E060E080E00E945209F60180818E7F89
:1013A0008083F80180818160808380818860808370
:1013B000F70180818E7F8083888180618883CDB7AB
:1013C000DEB7E8E00C942228E091370390913603D1
:1013D00026E0E91302C080E00895AE2FB0E02E9F12
:1013E000F0011124E85CFC4F3181361306C03081D6
:1013F000381303C03281341304C0FD013196E77005
:10140000E8CF81E0089581E08093E00080E280935E
:10141000D8001092C9008FE19EE40197F1F700C057
:10142000000087E090EBDC0180936E0390936F03E4
:10143000A0937003B093710388E19CE00FB6F89419
:10144000A895809360000FBE90936000FFCF0F932C
:101450001F93CF93DF93EB018A019091E9029430BF
:1014600079F58093E9008FEF9091E80095FD07C032
:1014700095ED9A95F1F7000081508111F5CF80919B
:10148000E80085FF1DC00E940209811114C08091EF
:10149000E80085FD06C08091E8008E778093E80023
:1014A000F2CF88818093F1000150110901151105D7
:1014B00011F02196ECCF8091E8008E778093E800C0
:1014C000DF91CF911F910F910895CF93DF93D82F84
:1014D000C92F48E050E0682F792F81E00E94270A49
:1014E00088E0ED2FFC2FAFEAB1E001900D928A95D4
:1014F000E1F7DF91CF910895BC0143E050E084E033
:101500000E94270A08959091340392FB222720F924
:10151000281779F080FB92F990933403609133039C
:101520007091340384E090E00E94062982E00E94DA
:10153000B8070895882381F063E282E290E00E9478
:10154000E82863E083E290E00E94E82869E184E211
:1015500090E00E94E82808956FEF82E290E00E94F8
:10156000E8286FEF83E290E00E94E8286FEFEFCF6A
:101570001F93CF93DF93962F122F632F8830D8F4C9
:101580009530C8F44530B8F4C42FD0E0CC0FDD1F3F
:101590002AE0929FC00DD11D112492E3899FC00DB6
:1015A000D11D1124CE0186960E94E828612FCE011C
:1015B00087960E94E828DF91CF911F910895AF92FE
:1015C000BF92CF92DF92FF920F931F93CF93DF933F
:1015D000A12CB12C00E0650110E013C0FE012591A3
:1015E00034914F2D612F802F0E94B80A2296F394D8
:1015F00085E0F812F3CF85E0C80ED11C1F5F1530CF
:1016000039F0E601CC0FDD1FCD5ADD4FF12CE6CFCE
:101610000F5F89E1A80EB11C0830E9F6DF91CF9188
:101620001F910F91FF90DF90CF90BF90AF900895E2
:10163000CF93DF93C6EBD1E060E0CE010E94E828B3
:101640002196C11584E0D807B9F7DF91CF910895AD
:1016500080E00E949A0A60E085E290E00E94E8281B
:101660000E94DF0A0E94180B81E00E949A0A0895E6
:1016700082E290E00E94D428833289F483E290E0F1
:101680000E94D428833059F484E290E00E94D42848
:1016900091E0893109F090E0892F8170089580E010
:1016A000FCCF0F931F93CF93DF93883030F56530D5
:1016B00020F5453010F5C42FD0E0CC0FDD1F2AE017
:1016C000629FC00DD11D112432E3839FC00DD11D37
:1016D0001124CE0186960E94D428082F10E0102FE6
:1016E0000027CE0187960E94D4289801282BC90193
:1016F000DF91CF911F910F91089580E090E0F8CF96
:10170000462F672F753038F4453028F4883018F4A8
:101710000E94510B089580E090E00895A0E0B0E0B1
:10172000E4E9FBE00C9407287C01009131038091EF
:101730003003082BC7E0D0E010E0C8010C2E02C037
:10174000959587950A94E2F780FD09C02197A8F73F
:10175000D12C8D2DCDB7DEB7E7E00C942328DC2EFD
:10176000B7018C2F0E94800B0E941A05019771F31C
:10177000F0CF0F931F93CF93FC01828100811181E1
:10178000882391F0662381F0C8010E948E0BC82F38
:10179000682FC8010E949C03B8018C2F0E94800B07
:1017A000CF911F910F910895C8010E94D303C82FB4
:1017B000F3CFCF93DF93D82FC92F0E948E0B6D2FBD
:1017C0007C2F0E94800B0E941A05DF91CF91089513
:1017D000FC0183819481892BC9F0818190818923C7
:1017E0008F3FA1F0808191810E94D90B282F929583
:1017F0009F70963091F060F4925F9F70923030F459
:1018000081E0203F79F030F4283E30F080E004C0E1
:101810009A5FF3CF243FD1F7089581E0283E18F076
:10182000213FF9CF0895089580912E0390913503BB
:10183000892B8093960190912F03992391F0892B06
:101840008093960120E088E991E0FC0130810196C7
:1018500031112F5F31E08E399307B9F721110E94C2
:10186000260448E050E06EEE72E086E991E00E94C6
:10187000C728892BA9F088E0E6E9F1E0AEEEB2E0F6
:1018800001900D928A95E1F7E091EC02F091ED0262
:10189000309731F00280F381E02D86E991E00995DF
:1018A0000895CF93C82F8823A9F08CEF8C0F813A2D
:1018B00098F4E8E9F1E08EE991E02191C217B1F1E5
:1018C0008E179F07D1F76C2F86E991E00E9443089D
:1018D0000E94140CCF91089580E28C0F883068F438
:1018E000C77021E030E001C0220FCA95EAF780916D
:1018F0002E03822B80932E03EBCF8BE58C0F83304E
:1019000038F42C2F2452330BC9010E94F707E2CF81
:10191000C85ACB31F8F6EC2FF0E0EE0FFF1FE35A78
:10192000FE4F808191810E941D08D4CF8C2F0E9490
:1019300011040E94140CC7CF882339F19CEF980F33
:10194000913A28F40E9411040E94140C089590E228
:10195000980F983050F4877091E001C0990F8A95E4
:10196000EAF7892F0E941E04EFCF9BE5980F933072
:1019700028F480E090E00E94F7070895885A8B31A0
:1019800020F480E090E00E941D0808950F931F93BB
:10199000CF93C82F00E010E0893311F400E510E088
:1019A0008C2F0E94510C0115110539F48C2F0E94C7
:1019B0009C0CCF911F910F9108958FE99FE00197A3
:1019C000F1F700C0000001501109EDCF882339F074
:1019D00090912E03892B80932E030E94140C08955E
:1019E000882321F00E941E040E94140C08950F9376
:1019F0001F93CF93DF93C62FD42F122F8823A9F0E4
:101A0000609323030E945D089093A2018093A1013B
:101A1000C77081E001C0880FCA95EAF70E94E60C02
:101A2000DF91CF911F910F91089580912303681347
:101A30003DC02091A1013091A2014FB7F89480914F
:101A4000B8019091B901A091BA01B091BB014FBF0B
:101A5000821B930B883C910548F56D130CC0812FB8
:101A60000E94C60CD77081E001C0880FDA95EAF7B2
:101A70000E94F00CD5CFC77001E0802F01C0880F05
:101A8000CA95EAF70E94F00C80E28D0F883050F47E
:101A90008D2F877001C0000F8A95EAF7802F0E9472
:101AA000E60CDDCF812F0E94C60CBACFC77081E053
:101AB00001C0880FCA95EAF7DBCF10922E03E8E940
:101AC000F1E086E0DF011D928A95E9F780E090E081
:101AD0000E94F70780E090E00E941D0810923503F5
:101AE0000E94140C08950E945D0D2FEF84E39CE08A
:101AF000215080409040E1F700C0000088E19CE068
:101B00000FB6F894A895809360000FBE9093600084
:101B1000FFCFAAE2B0E0EFE8FDE00C940B2887EAE3
:101B200091E0FC0101962091F100208321E08F3AA1
:101B30009207B9F78091A801893009F456C0C8F41A
:101B4000823009F4B3C0833009F482C0813071F16E
:101B50008091E80083FFE7C08091A7019091A801E0
:101B60009A3008F0E0C0E92FF0E0EF57F64D0C9402
:101B7000E0278A3009F489C08B3051F78091A701A2
:101B8000813231F78091AB019091AC01892B01F743
:101B90008091E800877F8093E8000E94E3088091AD
:101BA000A901809304010E945D0DD2CF8091A7010D
:101BB000813A71F68091E800877F8093E8008091F8
:101BC000AB019091AC01892B61F060E080E090E086
:101BD00070E00E948A088091E8008B778093E8008B
:101BE000B7CF68E08FEA91E0F3CF8091A70181320F
:101BF00009F0AECF8091AB019091AC018D7F892B24
:101C000009F0A6CF8091E800877F8093E80080915B
:101C1000E80082FF18C09091F3008091F2000297D3
:101C200031F48091F100813011F0863021F48091FF
:101C3000F1008093B7018091E8008B778093E800F2
:101C40000E94E30885CF8091E9028111E0CF80CF27
:101C50008091A701813A09F07BCF8091AB019091EF
:101C6000AC01892B09F074CF8091E800877F8093C5
:101C7000E8008091E80080FFFCCF80910401809310
:101C8000F1008091E8008E77D9CF8091A701813251
:101C900009F05ECF8091E800877F8093E8000E9482
:101CA000E3088091AA018093A30152CF8091A701FC
:101CB000813A09F04DCF8091E800877F8093E8005A
:101CC0008091E80080FFFCCF8091A301D8CF8038BD
:101CD00089F0823841F58091AB018F70873018F51B
:101CE0008093E9008091EB0085FB882780F91092B2
:101CF000E90006C08091A4019091D5029111826003
:101D00009091E800977F9093E8008093F100109203
:101D1000F1008091E8008E7723C0811116C0809178
:101D2000A901813011F18091E80083FF0AC0809100
:101D3000E800877F8093E8008091EB0080628093C9
:101D4000EB00AA96E3E00C942728823061F780919B
:101D5000A901882389F01092E9008091E800877F2B
:101D60008093E8000E94E308DECF81E0933009F021
:101D700080E08093D502EFCF8091AB018F702FEF81
:101D8000280F263080F68093E9002091EB0020FF99
:101D9000E2CF933031F48091EB0080628093EB00CE
:101DA000DACF9091EB0090619093EB0021E030E06E
:101DB000A90102C0440F551F8A95E2F74093EA003B
:101DC0001092EA008091EB008860E8CF8111ABCFE0
:101DD0001091A9011F778091E3008078812B809377
:101DE000E3008091E800877F8093E8000E94E30889
:101DF0008091E80080FFFCCF8091E30080688093B1
:101E0000E30083E0111101C082E08093E9028BCFEF
:101E10008058823008F087CF4091A9015091AA01E3
:101E20004C3D83E0580799F583E08A838AE28983F1
:101E30004FB7F894DE01139620E03EE051E2E32F25
:101E4000F0E050935700849120FF03C082958F707B
:101E50003F5F8F708A30C8F0895C90E08D939D93CE
:101E60002F5F243161F74FBF8091E800877F809317
:101E7000E8006AE270E0CE0101960E948A08809133
:101E8000E8008B778093E8004ECF805DE6CF8091AD
:101E9000AB019091AC01252F33272330310509F494
:101EA0004AC078F52130310509F479C08BE590E01E
:101EB000EEEAF1E02230310509F035CF2091E8005B
:101EC000277F2093E8002091AD013091AE01821769
:101ED000930708F49C0140E02115310509F064C026
:101EE000411162C08091E80082FDC9CF8091E90272
:101EF000882329F2853019F28091E80083FFF2CF20
:101F0000BECF2132310509F43BC02232310509F040
:101F10000ACF8330910508F006CFFC01EE0FFF1FBA
:101F2000E25EFE4F0190F081E02D855E9E4FDC0168
:101F30008C9190E011C0CA019927413089F082301C
:101F40009105B1F0892B09F0EECEEFE4F2E0E491D7
:101F50008E2F90E0EFE4F2E0009709F4E4CEAECFEC
:101F6000E3E3F2E0E4918E2F90E0E3E3F2E0F4CFDC
:101F7000EBE1F2E0E4918E2F90E0EBE1F2E0ECCFC8
:101F80008330910508F0CFCEFC01EE0FFF1FEC5D12
:101F9000FE4F0190F081E02D89E090E08FCF82E14B
:101FA00090E0E9E0F2E08ACF8091E902882309F429
:101FB00066CF853009F463CF8091E80083FD5FCF61
:101FC0008091E80082FD8ECF8091E80080FF84CF71
:101FD0009091F3008091F2002115310519F08830BD
:101FE000910550F041E0089709F040E08091E80049
:101FF0008E778093E80070CF44914093F100319642
:10200000215031090196E8CF803809F08CCE8091BB
:10201000E800877F8093E8008091A5018093F1001C
:1020200078CE811180CE1091A901123008F07BCEBC
:102030008091E800877F8093E8001093A5010E94BB
:10204000E3081123D1F084E08093E90242E061ECDF
:1020500081E00E94520942E261EC84E00E94520950
:1020600042E261EC82E00E94520942E260EC83E0CD
:102070000E9452098091E90256CE8091E30087FDCB
:10208000E2CF81E0E1CF67EE7EEF80E090E00E945A
:10209000062960E082E090E00E94E82860E083E0AA
:1020A00090E00E94E8281092300360E074E184E040
:1020B00090E00E94062960E086E090E00E94E82817
:1020C0006FEF87E090E00E94E82840E050E0BA011E
:1020D00088E090E00E94FA2860E08DE090E00E94A5
:1020E000E82840E050E0BA0188E190E00E94FA2838
:1020F00060E087E190E00E94E82840E050E0BA010B
:102100008CE190E00E94FA2860E070E080E290E0CC
:102110000E94062940E050E0BA0188E190E00E9468
:10212000FA2880E00E949A0A0E94280B40E050E0C2
:10213000BA018FE090E00E94FA2840E050E0BA0136
:1021400083E190E00E94FA2808950F931F93CF93A4
:10215000DF938B01D82FC92F0E94DB06A8016D2FBA
:102160007C2F88E090E00E94FA28DF91CF911F91A8
:102170000F910895E9E2F3E083E0808311828FEF0D
:10218000828386E98383148263E070E08FEF96E9AF
:102190000E94A5100895A4E0B0E0E1EDF0E10C94F8
:1021A0000C2880912D03833018F48F5F80932D03CA
:1021B0008091290390912A03A0912B03B0912C03C5
:1021C000BC01CD010E94A5102496E2E00C942828C1
:1021D000A4E0B0E0EEEEF0E10C940C2880912D0329
:1021E000882319F0815080932D03809129039091C9
:1021F0002A03A0912B03B0912C03BC01CD010E94B6
:10220000A5102496E2E00C94282860912903669595
:1022100070E04BE050E088E091E00E94BA28892B02
:1022200019F481E0809326030E945D089093DE02FA
:102230008093DD020895A5E0B0E0E1E2F1E10C94C5
:10224000FF278091290380FD0AC0E7E6F2E01182B2
:1022500010821282339622E0EA3CF207C1F78090A6
:10226000D0029090D1028114910409F465C080914C
:10227000D402811161C050902C03A12CB12C662492
:102280006394712C2091270330912803C3010A2CF9
:1022900002C0880F991F0A94E2F782239323892BA7
:1022A00009F43FC0F401E590F490E114F10409F45D
:1022B00043C045E050E0B701CE0101960E94B1282D
:1022C00089818F3F71F12A8190E0280F392F311DCC
:1022D0002232310514F021E230E06901CC0CDD1C22
:1022E000C20ED31E960129593D4F69018C01000F82
:1022F000111F080F191F09591D4F0C151D0520F03E
:1023000055E0E50EF11CD5CF452D36E9351508F41D
:1023100046E998016C818B810E944F060D5F1F4F2B
:10232000ECCF82E0880E911C9FEFA91AB90A29E030
:10233000A216B10409F0A6CF559A3BB13F7D2BB14F
:1023400020624FB7F89487E692E0FC010196508135
:1023500068E02BB9000000C057FF3BB9550F0000E3
:1023600000C000C000C03BB900C06A9591F752E0C0
:102370008A3C950751F74FBF8FE594E00197F1F73D
:1023800000C000002596EFE00C941B28A0E0B0E010
:10239000ECECF1E10C94FE27FC016280448081E0CA
:1023A0008483E3EEF3E07490E2E6F4E0E4910091DC
:1023B0002C030695015810E0000F111F012F112763
:1023C000C0ECD1E027E6C22E22E0D22E35E6832EE5
:1023D00032E0932EAA24AA94B12C55245A94E719DA
:1023E000EE2EF12C82E0861530F080912A0388834E
:1023F00080912B038983411019C01B821A824A8164
:10240000473908F046E99601698188810E944F06A4
:10241000259683E0C80ED11C8C169D0619F70E94E4
:102420001B11CDB7DEB7E0E10C941A288B8188230D
:10243000E9F081508B83589EC00111246C8170E0BB
:102440000E94B827FB01FF27ED51FC4F8491E82F34
:10245000E7195E9EC0011124B7010E94B827809140
:102460002C03689FB00111247A83C9CF0E94A12850
:10247000B5010E94CC27801791070CF0C0CF82E0F5
:10248000861588F40E94A128B5010E94CC27888374
:102490000E94A12820912B032695622F70E00E94B4
:1024A000CC27280F29831A8280912C03893C20F0A5
:1024B00088EC8C838B83A3CF8431D8F784E1F9CF68
:1024C000EF92FF921F93CF93DF93EC0187E6E82E04
:1024D00082E0F82E10E040912C03473908F046E9DD
:1024E0008C81970160912B03810F0E944F06195F29
:1024F00083E0E80EF11C173E71F70E941B119A81D0
:102500008C8190FF08C08F5F8C83DF91CF911F91EA
:10251000FF90EF9008958150F7CFA0E0B0E0E3E99D
:10252000F2E10C940628FC018281DD24D39480FF23
:1025300002C0DD24DA9407E612E0C0E0D0E0F80142
:1025400011821082128294E0E92EF12CC12C80912C
:1025500066028C0D8232ECF161E20E94AA27892F7B
:10256000082E000C990B8C179D07A9F480912C0361
:102570008E9DA0018F9D500D112455954795559521
:102580004795473908F046E9980160912B038091FF
:102590002A030E944F06CD0CF1E0EF1AF108E11476
:1025A000F104A9F621960D5F1F4FC132D10539F60E
:1025B0000E941B118091660291E0D9120EC08823FF
:1025C00091F0815080936602CDB7DEB7E8E00C94BD
:1025D000222887FFC5CF8F5DC3CF90E00196BE0153
:1025E0000E94CC27EFCF80E2EDCF0F931F93CF93C4
:1025F000DF93C7E6D2E0FE01118210821282339689
:1026000082E0EA3CF807C1F700E010E08091650243
:10261000082E000C990B08171907A4F180910701E7
:10262000082E000C990B8017910764F140912C0340
:10263000473908F046E99E0160912B0380912A03F7
:102640000E944F060F5F1F4F239601321105F1F6CE
:102650000E941B118091060190916502980F909342
:10266000650220910701280F20930701121614F428
:1026700090321CF0819580930601DF91CF911F91DC
:102680000F910895198218821A82DCCFAEE0B0E073
:10269000ECE4F3E10C9406288D879E87AD85BE851A
:1026A00014961C91212F30E0D9010E9470299B01C2
:1026B000AC010E943B2969837A838B839C83E0E28F
:1026C000F0E0E11BF109A5E5B0E09B01AC010E943F
:1026D0003B2969877A878B879C879F01DF010E944E
:1026E000ED279B01AC010E9446296D837E838F8379
:1026F00098879B01AC0189819A81AB81BC81280FAD
:10270000391F4A1F5B1F69857A858B859C850E94CE
:102710004E29022F30E00A32E0F5C901880F991FD7
:10272000820F931F95958795182F109537E6C32E26
:1027300032E0D32EF12C85E5E82EE01A8E2DF1FC47
:10274000802F412F173908F046E9960160912B033D
:102750000E944F06F394B3E0CB0ED11CE1E2FE12CF
:10276000EDCF0E941B11AD85BE8514969C9181E032
:10277000992319F0903219F48FEF8093050180911D
:102780000501890FED85FE8584832E96E8E00C9483
:10279000222885E590E0DC01A21BB30BCD01880F58
:1027A000991F8A0F9B1F97FFBDCF0196BBCF9091BA
:1027B000290390FF0CC0E7E6F2E081836083428347
:1027C000339692E0EA3CF907C1F70E941B11089585
:1027D000A3E0B0E0EEEEF3E10C940C289091290315
:1027E00090FF0DC0473908F046E99E012F5F3F4F2B
:1027F0000E944F064B8169818A810E94D7132396DC
:10280000E2E00C942828CF93DF93EC01EC81F0E018
:10281000ED51FC4F4491E9E2F3E0628181810E9435
:10282000E8138C818F5F8C83DF91CF910895CF93D4
:10283000DF93EC01E9E2F3E0438162818C810E9445
:10284000E8138C818F5F8C83DF91CF910895A7E08F
:10285000B0E0EDE2F4E10C94FF27E82E762EF42EA2
:10286000622E9091290390FF32C0E92FE695AE2F9A
:10287000B0E0A65DBE4F8C91809325039E7F923081
:1028800051F540932C0386E9841708F446E99E012C
:102890002F5F3F4F672D8E2D0E944F064B81698120
:1028A0008A810E94D713E0922A0370922B03F09240
:1028B0002C03662061F08091290390912A03A09156
:1028C0002B03B0912C03BC01CD010E94A5102796CB
:1028D000EFE00C941B28823019F4F0902C03E3CF26
:1028E000863019F4E0902A03DECF8930D9F389319C
:1028F000D1F6E9519E2F9170592EE695F0E0ED51F9
:10290000FB4FE4910E2F10E087E6C82E82E0D82E10
:10291000A12CB12C91E2892E912CC501B4010E9409
:10292000B8278E2D511019C0860F4F2DA6E9AF156F
:1029300008F446E99601672D0E944F06A00EB11ECD
:10294000B3E0CB0ED11C8AECC81682E0D80629F77A
:10295000F0922C030E941B11A6CF861BE6CFA4E0A9
:10296000B0E0E5EBF4E10C940C289091290390FF82
:1029700034C08823B1F18932B0F58F77880F9091F8
:1029800029039170892B80932903662361F080913C
:10299000290390912A03A0912B03B0912C03BC0131
:1029A000CD010E94A51060912903669570E04BE06F
:1029B00050E088E091E00E94BA28892BB1F0109293
:1029C000260381E08093E00220E040912C03609197
:1029D0002B0380912A030E9427142496E2E00C9492
:1029E000282881E0CBCF88E2C9CF0E940511E9CF2A
:1029F0008091290386958F5F893208F081E061E03C
:102A00000E94AF1408959091290396958FEF890F36
:102A1000913009F488E261E00E94AF140895E9E280
:102A2000F3E080818160808360E086950E94AF142E
:102A300008959091290390FF08C09695981728F063
:102A4000961718F40E94F814089561E00E94AF14DC
:102A50000895A4E1B0E0EFE2F5E10C94FC278D8746
:102A60009E87AD85BE859C9111968C91119713968A
:102A70002D913C911497232B09F413C189238F3F87
:102A800009F40FC161E0CD010E94B90B4C01ED8545
:102A9000FE85A281815A92454F9708F07BC0840140
:102AA000F0EA0F27F2E51F27AA2309F490C38091CB
:102AB0002203882309F4D9C110922203480121E09E
:102AC00030E040E050E060E070E080E090E0082D11
:102AD0000E943328E09102032E2BE09103033E2B4A
:102AE000E09104034E2BE09105035E2BE091060379
:102AF0006E2BE09107037E2BE09108038E2BE09173
:102B00000903E92B2093020330930303409304034A
:102B100050930503609306037093070380930803A3
:102B2000E0930903AA2309F453C61092230397E7FD
:102B300089169CE7990609F4CBC682E0A8E78A16B5
:102B4000ACE79A0609F4C5C6FAE58F16FCE79F06BE
:102B500009F4E8C608F0C9C631E083163CE79306DD
:102B600009F4DEC643E084164CE7940609F4D2C6A5
:102B700081148CE7980609F038C60E945D0DBFEFFE
:102B8000E4E3FCE0B150E040F040E1F700C00000B9
:102B90000E94030AAA2309F40FC32FEF821691049F
:102BA00009F008F482C039E583163CE7930609F47E
:102BB00060C010922203C40197578038910508F035
:102BC0002CC3182D103108F05AC08FEF93E00E94EB
:102BD000D428811154C056EB652E772473941111BB
:102BE000BAC31A821982FE01339686E0DF011D9274
:102BF0008A95E9F74AE0242E4301BFEF8B1A9B0A1E
:102C0000C3010E94D42889831A828823C1F18130AC
:102C100009F0D4C383010E5F1F4FC4010E94D42862
:102C20008A83882361F19FEF980F933008F0A2C345
:102C3000E3E06E0E711CC8010E94D4288B838823A8
:102C4000F1F01C828E010F5F1F4FD8018C918823F9
:102C500099F2813009F0EDC311969C91119712966B
:102C60008C91913009F0ACC30E5F1F4F0E94C60CCF
:102C7000ADC38091220391E0892780932203809144
:102C800032038770882369F0AD85BE8512968C91DA
:102C9000882339F08091340382FF03C082E00E94D0
:102CA000B8076496E2E10C941828809122038823E7
:102CB00009F4D5C01092220340EC8416910408F464
:102CC00058C021E030E040E050E060E070E080E09B
:102CD00090E08401005C11090E943328E0911A03FE
:102CE0002E2BE0911B033E2BE0911C034E2BE09119
:102CF0001D035E2BE0911E036E2BE0911F037E2BC4
:102D0000E09120038E2BE0912103E92B20931A03FD
:102D100030931B0340931C0350931D0360931E03C9
:102D200070931F0380932003E0932103AA2309F4E7
:102D3000ACC210922303C4019057839708F4F4C3E4
:102D4000F6E18F16FCE79F0609F0F1CE80912E0385
:102D50008A7A91E0811101C090E09093240369E2A6
:102D6000811165E386E991E00E9443080E94140CFA
:102D700086CF80E888169104E0F58401005411099B
:102D80000034110508F09BCE21E030E040E050E037
:102D900060E070E080E090E00E943328E0910A0358
:102DA0002E2BE0910B033E2BE0910C034E2BE09178
:102DB0000D035E2BE0910E036E2BE0910F037E2B33
:102DC000E09110038E2BE0911103E92B20930A036D
:102DD00030930B0340930C0350930D0360930E0349
:102DE00070930F0380931003E09311031092230359
:102DF000A4CE21E030E040E050E060E070E080E010
:102E000090E08401005811090E943328E0911203D8
:102E10002E2BE09113033E2BE09114034E2BE091F7
:102E200015035E2BE09116036E2BE09117037E2BAA
:102E3000E09118038E2BE0911903E92B20931203E4
:102E400030931303409314035093150360931603B8
:102E50007093170380931803E0931903C7CF90E48E
:102E60008916910408F066C0840120900203B09195
:102E70000303B987E0910403EF87F0910503F88B12
:102E8000B0910603B98BE0910703EA8BF091080338
:102E9000FB8BB0910903BC8B21E030E040E050E0B7
:102EA00060E070E080E090E00E943328322E432EF4
:102EB000542E652E762EB72FF82FE92FA22CA222A2
:102EC000B984B322CF84C422D888D522E988E622E7
:102ED000FA88F7220B8908231C8919230E944C28A1
:102EE00009F02FC230944094509460947094B0953F
:102EF000F095E0953220A9854A22AF855A22A8890B
:102F00006A22A9897A22AA89BA23AB89FA23AC89D1
:102F1000EA2330920203409203035092040360922A
:102F2000050370920603B0930703F0930803E09340
:102F30000903A5CEE0E88E16910408F068C0209041
:102F40000A03F0910B03F987B0910C03BF87E0915E
:102F50000D03E88BF0910E03F98BB0910F03BA8B40
:102F6000E0911003EB8BF0911103FC8B21E030E03A
:102F700040E050E060E070E080E090E084010054C8
:102F800011090E943328322E432E542E652E762EA0
:102F9000B72FF82FE92FA22CA222B984B322CF8415
:102FA000C422D888D522E988E622FA88F7220B893C
:102FB00008231C8919230E944C2809F0B7CE3094AD
:102FC0004094509460947094B095F095E0953220C0
:102FD000A9854A22AF855A22A8896A22A9897A221C
:102FE000AA89BA23AB89FA23AC89EA2330920A036F
:102FF00040920B0350920C0360920D0370920E03EB
:10300000B0930F03F0931003E093110338CE20EC3C
:103010008216910408F068C020901203B091130347
:10302000B987E0911403EF87F0911503F88BB09105
:103030001603B98BE0911703EA8BF0911803FB8B11
:10304000B0911903BC8B21E030E040E050E060E03B
:1030500070E080E090E08401005811090E9433285C
:10306000322E432E542E652E762EB72FF82FE92FB1
:10307000A22CA222B984B322CF84C422D888D5221C
:10308000E988E622FA88F7220B8908231C8919238C
:103090000E944C2809F04ACE309440945094609499
:1030A0007094B095F095E0953220A9854A22AF85BD
:1030B0005A22A8896A22A9897A22AA89BA23AB89C5
:1030C000FA23AC89EA233092120340921303509200
:1030D00014036092150370921603B0931703F093D4
:1030E0001803E0931903CBCD20901A03E0911B0342
:1030F000E987F0911C03FF87B0911D03B88BE09125
:103100001E03E98BF0911F03FA8BB0912003BB8B58
:10311000E0912103EC8B21E030E040E050E060E002
:1031200070E080E090E08401005C11090E94332887
:10313000322E432E542E652E762EB72FF82FE92FE0
:10314000A22CA222B984B322CF84C422D888D5224B
:10315000E988E622FA88F7220B8908231C891923BB
:103160000E944C2809F0E2CD309440945094609431
:103170007094B095F095E0953220A9854A22AF85EC
:103180005A22A8896A22A9897A22AA89BA23AB89F4
:10319000FA23AC89EA2330921A0340921B0350921F
:1031A0001C0360921D0370921E03B0931F03F093E3
:1031B0002003E093210363CDBFEF8B16910411F040
:1031C00008F0C1C0E0E48E16910490F5840121E07E
:1031D00030E040E050E060E070E080E090E00E948D
:1031E0003328A0900203A222B0900303B322C09020
:1031F0000403C422D0900503D522E0900603E62202
:10320000F0900703F72200910803082310910903A7
:1032100019230E944C2809F432CDF401E851FC47EF
:10322000E730F10508F082CDE557F64D0C94E02724
:10323000F0E88F169104B8F521E030E040E050E06E
:1032400060E070E080E090E08401005411090E9489
:103250003328A0900A03A222B0900B03B322C0909F
:103260000C03C422D0900D03D522E0900E03E62279
:10327000F0900F03F722009110030823109111031F
:1032800019230E944C2809F4FACCE6E18E16ECE7EB
:103290009E0609F01AC280912403811114C289E2AA
:1032A0000E94110463CD20EC8216910428F521E0E0
:1032B00030E040E050E060E070E080E090E08401C9
:1032C000005811090E943328A0901203A222B09046
:1032D0001303B322C0901403C422D0901503D52247
:1032E000E0901603E622F0901703F72200911803EE
:1032F000082310911903C4CF21E030E040E050E0F2
:1033000060E070E080E090E08401005C11090E94C0
:103310003328A0901A03A222B0901B03B322C090BE
:103320001C03C422D0901D03D522E0901E03E62288
:10333000F0901F03F722009120030823109121032E
:103340009FCFA11138CCF401E851FC47E730F105DB
:1033500008F09BCF69CF611434E0730609F48FCC79
:10336000C3010E94D428D30111963D018111F3CFEE
:10337000115035CC8430C1F432E0832E912CC80139
:103380000F5F1F4F0E94D428E1E0F0E0EC0FFD1F1B
:10339000E80DF91D8083882309F471CC8C3731F452
:1033A000FE01E80DF91D128238014CCCFFEF8F1A97
:1033B0009F0A27E08216910411F761CC340142CCB8
:1033C000923039F40E5F1F4F0E94510C0F5F1F4F58
:1033D0003CCC933029F40E5F1F4F0E949C0CF6CF1B
:1033E000943019F00F5F1F4FF1CF0E5F1F4F20E099
:1033F00030E0A8014F5F5F4F8053990B8A309105F1
:1034000060F02115310511F38FE99FE00197F1F785
:1034100000C0000021503109F4CF229EB001239E4C
:10342000700D11249C01260F371FF80181818A013C
:10343000E0CFE82FF0E0E35CF94F3490282F269599
:103440002695269530E0F901E35DF94F9491877058
:10345000F901E35EF94F8490912C082E02C09594F7
:1034600087940A94E2F7A1E08A229924F901E35FA4
:10347000F94F4490512C082E02C0559447940A9459
:10348000E2F7B1E04B225524292F30E002C03595F8
:1034900027958A95E2F720FF0AC081EE0E94510C21
:1034A0008928D1F4832D0E94C60C81EE12C0892890
:1034B00049F4832D0E94C60C4114510409F486CFAF
:1034C0008CE2D4CB86EE0E94510C832D0E94C60C58
:1034D00086EE0E949C0CF0CF86EE0E94510C832D4C
:1034E0000E94C60C86EE0E949C0CDFCF26E241EEC5
:1034F00061EE8A2F0E94F70CC2CB27E245EE65EE03
:10350000F8CF26E241EE60EEF4CF27E245EE64EE1E
:10351000F0CF26E241EE62EEECCF27E245EE66EE1A
:10352000E8CF28E241E0EBCF84E090E00E94E2287F
:103530009093340380933303F401E150F047E23277
:10354000F10520F4EE56F64D0C94E02780913303FC
:10355000816080933303609133037091340384E07E
:1035600090E00E9406290E945D0D89CB8091340372
:10357000886080933403EFCF809133038260E9CF7A
:10358000809133038460E5CF809133038860E1CF7D
:10359000809134038160EDCF809134038260E9CF64
:1035A000809133038061D5CF809133038062D1CF86
:1035B000809133038064CDCF0E945D0D80913303F1
:1035C0008068C7CF809133038C60C3CF8091340370
:1035D0008360CFCF809133038E7FBBCF8091340344
:1035E000877FC7CF809133038D7FB3CF8091330323
:1035F0008B7FAFCF80913303877FABCF8091340334
:103600008E7FB7CF809134038D7FB3CF809133030A
:103610008F7E9FCF809133038F7D9BCF809133032B
:103620008F7B97CF0E945D0D809133038F7791CF71
:1036300080913303837F8DCF809134038C7F99CF2A
:103640008091330382FB992790F921E0922790FB28
:1036500082F990FB83F97DCF80913403982F909568
:1036600091708E7F892B90FB81F983CF90913303EA
:10367000892F8F7B96FF80646CCF0E945D0D9091A7
:103680003303892F97FB87F9805863CF61E08EE081
:1036900090E00E94E8285FCF60E0F9CF909133037B
:1036A000892F8F7E94FF806154CF90913303892FAF
:1036B0008E7F90FF81604DCF90913403892F877F5B
:1036C00093FF886056CF85E3EBCD80912E03827205
:1036D000F401E052F847E531F10508F079C0EC5407
:1036E000F64D0C94E0278091290380FF18C08E7F4F
:1036F000809329038091290390912A03A0912B03A1
:10370000B0912C0389879A87AB87BC87BC01CD0118
:103710000E94A510109226030E941B11B0CA81605E
:103720008093290361E086950E94AF14A8CA43E004
:1037300055E168EF74E10E941407A1CA48EF54E113
:1037400063E075E1F8CF42EC50E268EB70E2F3CF52
:1037500048EB50E262EC70E2EECF49ED50E26CECE7
:1037600070E2E9CF4CEC50E269ED70E2E4CF43EF58
:1037700050E266EE70E2DFCF46EE50E263EF70E2B9
:10378000DACF48EE50E16BEC70E1D5CF4BEC50E175
:1037900068EE70E1D0CF61E081E0C6CF65E082E005
:1037A0000E9419156CCA68E086E0FACF6EE089E0E5
:1037B000F7CF64E18FE0F4CF67E185E1F1CF61E01D
:1037C00088E1B2CF62E289E1EBCF68E283E2E8CF41
:1037D000B7E78B16BCE79B0609F483C082E0E8E7F5
:1037E0008E16ECE79E0609F47DC0ED85FE8582818C
:1037F00080809180882309F499C0C4010E948E0BB7
:10380000182F682FC4010E949C03B401812F0E94CD
:10381000800B0E941A058C01AD85BE8512968C9096
:10382000129715967C9072942FE072228091320349
:1038300087708823F1F0682C8820E1F0812F807F49
:10384000803451F080E2800F883098F0711004C00D
:10385000812F807E803269F08091340382FF09C01D
:1038600082E00E94B80780913203877066246394D7
:103870008111612C812F82958F70883009F440C1AD
:1038800008F07BC0843008F056C0B12FBF709B2E6B
:10389000823008F483C0107F103219F0929480EFC8
:1038A0009822002309F4B1C0013009F4F0C0882047
:1038B00009F4FAC0772009F4F0C0AD85BE851596ED
:1038C0008C91159780FF80C08F7015968C93E5C002
:1038D00081E00E949C0743E062E081E00E94D607FD
:1038E000CEC981E00E94A807F6CF9BE589169CE728
:1038F0009906D1F0ACE58A16ACE79A0609F075CFC7
:103900008091340382FB882780F991E089270E9407
:10391000830A6BCF6FEF7FEF80E090E00E94062973
:103920000E94730D81E0F3CF80E0F1CFC4010E94CB
:10393000D303182F6ACF843009F4C7C06620B9F0CA
:103940008091320380FD13C0ED85FE85128285953E
:10395000859585950E949C078D859E850E942915D9
:10396000809132038595859585950E94A80760E032
:103970008D859E850E94B90B94C9893009F431C1A7
:103980008A5F8F708230D0F6023F09F03BC1812FF1
:103990008F71811034C10E949C07DFC0103118F074
:1039A000929490EF99228820B9F0992069F080E2F2
:1039B000800F883010F0011109C080912E038929F1
:1039C00080932E030E94140C802F2FC0809135030A
:1039D000892980933503F6CF802F0E949C0C992073
:1039E00009F4ACCF80E2800F883010F0011104C0E0
:1039F000892D0E941E0406C0909480913503892170
:103A0000809335030E94140C99CF2091340322FD3A
:103A100016C0882069F0992039F080912E038929F9
:103A200080932E030E94140C80E00E94510C86CFDC
:103A300080E00E949C0C992009F480CFD9CF882087
:103A4000A1F090912F03892D892B711003C00E9442
:103A5000E60C74CFE1E07E12FACF22FF6FCF891718
:103A600009F46CCF80932F0369CF711006C00E94B8
:103A70002604892D0E94F00C61CFF1E07F1609F435
:103A80005DCF892D0E94F00C0E94260457CF88201C
:103A900031F025E0271508F451CF892DD8CF34E037
:103AA000371508F44BCFE5CF772019F3093349F4E4
:103AB000BFEFE7EEF3E0B150E040F040E1F700C0C7
:103AC0000000802F0E949C0C39CF812F869586950F
:103AD0008370882361F0813009F030CFC801937082
:103AE000811002C080E090E00E941D0827CFC8012D
:103AF0009370811002C080E090E00E94F7071ECF13
:103B0000812F8370811136C0811027C0402F4295CC
:103B100046954770440F440F802F8F70042E01C0CC
:103B2000880F0A94EAF70071002341F02FE030E09B
:103B300001C0220F4A95EAF7022F009516951695B7
:103B40001370123091F0133071F020913003113066
:103B500049F0802B82230E9499030E941B070E9438
:103B60000E07ECCE822B802BF6CF802B909130036A
:103B70008927F1CF882051F110FFEFCF402F4295D8
:103B800046954770440F440F802F8F70042E01C05C
:103B9000880F0A94EAF70071002341F02FE030E02B
:103BA00001C0220F4A95EAF7022F00951695169547
:103BB0001370123089F0133069F020913103113005
:103BC00041F0802B82230E949707C7CF823028F2D2
:103BD000D5CF822B802BF7CF802B90913103892773
:103BE000F2CF1F70882039F0812F0E949C07802F10
:103BF0000E94E60CB2CF802F0E94F00C812F0E9411
:103C0000A807ABCF033F70F4003FB9F0013FB9F113
:103C1000882009F45BC0772009F455C0802F0E94EA
:103C2000510C9BCF033FD9F0043F29F18110F3CF12
:103C300071105AC0812F8F71E2CF882069F024E083
:103C4000271508F48ACF1F7181E090E0012E01C092
:103C5000880F0A94EAF7C1CF35E07316F2CF80E0FF
:103C6000882009F4B0CF1F7181E0012E01C0880FB8
:103C70000A94EAF7A8CF8091340382FD06C0812F11
:103C80008F71882009F4BBCF86CE882089F01F7100
:103C9000812F0E949C078091340382FF07C048E077
:103CA000149FC0011124836080933203812F73CE4F
:103CB00081E00E94B80781E0871508F04ECF82E0CE
:103CC0000E94B8074ACF812F8F7165CE772009F403
:103CD000B1CF093349F49FEFA7EEB3E09150A04074
:103CE000B040E1F700C00000802F0E949C0C35CF4F
:103CF0001F93CF93DF9380916D03803108F04CC008
:103D000080916A03882309F447C08091370320918A
:103D100036033091680360916903C0916B03D091C1
:103D20006C03732F76232817B9F190E0209709F4DC
:103D300043C016E07F3F09F43FC0189FF001199F70
:103D4000F00D1124DF01A85CBC4F11964C91119726
:103D500046132CC04C91431329C012964C911297D4
:103D600041111EC013964D915C914C1B5D0B483C5C
:103D70005105E0F480916D038F70806180936D0335
:103D8000E35CFC4F80818F708061808388E693E0E4
:103D90000E9429150E940704DF91CF911F91089579
:103DA0000196877099272813C8CFF6CF01968770A0
:103DB00099272813BFCFF0CF01968770B4CFABE01F
:103DC000B0E0E5EEFEE10C9403288C0185E0F801FB
:103DD000DE01179601900D928A95E1F7F801928025
:103DE000C380D48088E6A82E83E0B82E8091680333
:103DF0009091690320916B0330916C03211531057B
:103E000009F403C1482F49234F3F09F4FEC0E09055
:103E10006A03A601421B530BEE2009F4C9C0F090BF
:103E20006D03483C510508F0A3C0B1805FE05F1509
:103E300008F462C09B1114C09081981311C09110B6
:103E40003FC08F2D8F70806180936D0388E693E073
:103E50000E94291580916D03F8018583F12C29C0FA
:103E6000FF80C114D10451F18F2D8B218F3F31F18F
:103E7000911026C040E06B2D8F2D0E94E40940E098
